:10000000C0060020250100002101000021010000A0
:1000100000000000000000000000000000000000E0
:1000200000000000000000000000000021010000AE
:10003000000000000000000021010000210100007C
:100040002101000021010000210100000D0C000031
:10005000210100002101000021010000911D00008C
:100060002101000021010000210100002101000008
:10007000210100000000000000000000210100003C
:1000800021010000210100002101000021010000E8
:10009000210100000000000000000000210100001C
:1000A00021010000210100002101000021010000C8
:1000B0000000000010B5064C2378002B07D1054B3B
:1000C000002B02D0044800E000BF0123237010BDC4
:1000D0000000002000000000781F0000084B10B551
:1000E000002B03D00749084800E000BF0748036819
:1000F000002B00D110BD064B002BFBD09847F9E731
:100100000000000004000020781F0000781F00009D
:100110000000000010B5014B984710BD010400001D
:10012000FEE70000F8B5234A234B9A4209D0224B40
:10013000204A03E011681960043304321F498B42DE
:10014000F8D31F4B02E000221A6004331D4A934289
:10015000F9D31D4AFF211D4B8B439360FD3990233A
:100160005B001B4AD1501B4AD3780325AB430224C2
:100170002343D370D3780C27BB4308263343D37073
:10018000154B987B30229043202210439873997B23
:10019000B943314399739A7BAA4322439A730F4A16
:1001A000516880230B4353600D4B98470D4B984784
:1001B000FEE7C046781F000000000020000000207D
:1001C00000000020BC02002000ED00E00000000064
:1001D00000700041005000410048004100400041D3
:1001E000D51D00009D1D000010B5084A936920210F
:1001F0000B439361064A074B5A80074B984702000E
:1002000006490748074B984710BDC0460004004008
:1002100004400000000C0040090C000000140040E5
:10022000A00200207D070000F0B5C64600B5C02240
:10023000D205102353619360254B26499962C02152
:1002400009068C4699624420195C0127B9430126AE
:100250003143C9B219543221585C0F25A8430324F5
:10026000A04644462043C0B25854202050619060BC
:10027000194898626046986245208446185CB843E5
:100280003043C0B264461855585C363C2040302498
:10029000A44664462043C0B258540E3151600F4A00
:1002A0009A620F4A9A624622995C042081439954CB
:1002B000995CB9433143C9B2995433215A5CAA437A
:1002C00040460243D2B25A5404BC9046F0BDC046E8
:1002D0000044004110000040200000404000024067
:1002E000000002C0044A136A04210B431362034A4C
:1002F000034B5A807047C046000400401440000081
:10030000000C004010B5044B984704490448054BC5
:100310009847054B984710BDE502000000080042D1
:1003200088020020A905000029020000F0B5C64699
:1003300000B5C024E40580225204A2601C4B802733
:10034000FF059F621B49996262615820195C042273
:10035000904691431954195C0126B1430125294364
:10036000C9B219541C38195C0B32914306229446C9
:1003700062461143C9B2195480218904A1609F6269
:100380000D4F9F62616159215C5C424694435C540D
:100390005A5CB2432A43D2B25A541A5C4A390A40D0
:1003A00060210A43D2B21A5404BC9046F0BDC04644
:1003B00000440041000100C0000200C0064BDA69A1
:1003C00020210A43DA615A6920310A435A61034AFB
:1003D000034B5A807047C0460004004006400000AE
:1003E000000C004010B5034B9847034B9847034B54
:1003F000984710BDBD0300000D0A00002D0300004A
:1004000070B5514B9847514B40201A5C01218A43EB
:100410001A5401301A5C8A431A54C022D2053D385E
:10042000506190604A489862C02000069862422558
:100430005C5D8C435C55082454619460454C9C621F
:10044000986201355C5D8C435C55802454619460F6
:10045000414C9C62986204355C5D8C435C55802401
:100460006400546194603D4C9C62986201355C5D0F
:100470008C435C558024A40054619460384C9C6289
:10048000986201355C5D8C435C558024E4005461C6
:100490009460344C9C62986201355C5D8C435C5581
:1004A00080242401546194602F4C9C6298624B24F8
:1004B000185D884318550334185D88431855013476
:1004C000185D88431855802040025061906080205C
:1004D000C0059862254C9C6206355C5D8C435C557A
:1004E0008024A402546194609862214C9C6201357E
:1004F0005C5D8C435C558024E40254619460986296
:100500001C4C9C6201355C5D8C435C55802424034B
:10051000546194609862184C9C6201355C5D8C4318
:100520005C558024E403546194609862134A9A6293
:1005300056201A5C8A431A54114B9847114B98471E
:10054000114B984770BDC046E10A000000440041CD
:10055000040000400800004080000040000100400E
:10056000000200400004004000080040010000C0FC
:10057000020000C0040000C0080000C0400000C02D
:1005800005030000E9010000E5030000EFF310831C
:10059000036072B6BFF35F8F7047BFF35F8F03686E
:1005A00083F310887047000070B504000D00002828
:1005B00017D0002913D0012040220B490B4B98473C
:1005C0006560201D29000A4B9847002806DB094B6F
:1005D000A382094B2361094BE360002070BD00201A
:1005E000EAE70020E8E7C046401E0000790A000064
:1005F000310C00000080FFFF850600004906000066
:1006000030B587B004000D00002815D0002911D0A6
:100610000120B32209490A4B98472B6803936B6862
:100620000493AB6801930593201D03A9054B9847DC
:1006300007B030BD0020ECE70020EAE7401E0000D4
:10064000790A00002D0E000070B584B004000E0081
:100650001500431E9841C0B2A3220749074B984793
:1006600020000C38002302930196039501A9044B46
:10067000984704B070BDC046401E0000790A0000D3
:100680000106000070B584B004000E001500431E82
:100690009841C0B287220749074B984720000C3881
:1006A000029600230193039501A9044B984704B0D7
:1006B00070BDC046401E0000790A0000010600001F
:1006C000F8B50668002E02D0330000250CE0104B70
:1006D000984718E09F68BC466444A41A01348F68A8
:1006E000BC420BD21D001B68002B07D05C689442F3
:1006F000F0D8A41A9F68BC466444F0E7B34203D024
:100700002800044B9847F8BD014B9847FBE7C046CB
:10071000990A0000C50A0000F8B50500446903699C
:100720005E1C0661037EDB0702D4037E9B070AD5AD
:100730002B7E02221343DBB22B76F8BD6F69E36890
:10074000200098473C00002CF7D06368F31AA26899
:100750009342F2D32F0014373800064B9847237C7E
:10076000012BEBD16660320021003800024B984724
:10077000E4E7C046CD0A0000C106000070B50400E1
:100780000D00002812D000290ED001203B2208497C
:10079000084B984729002000074B98470023236106
:1007A000064B2360002070BD0020EFE70020EDE73E
:1007B0005C1E0000790A0000AD0B00001907000064
:1007C00010B50100002001E0013040B203280FDC29
:1007D0004201094B9B185A788A420BD04301064CC0
:1007E0001B5D002BF0D10F330B409342ECD101E0A5
:1007F0000120404210BDC0461C0000200020704770
:1008000070B504000D00084B98474201074B9B1838
:100810009B78032B01D0002070BD044B981883698E
:10082000290020009847F7E7C10700001C000020BE
:10083000F0B587B005000F0001924A4B98470400BD
:100840004601494A9619002F51D113004201002058
:10085000F070D35C002B0ED06201434B9B18012239
:100860009A706401404B1C19E369E178019A2800F1
:10087000984707B0F0BDB3780C243457032B08D049
:1008800032000C3270780021F36998470223B3706C
:10089000EFE7707832000C320121F36998470028A5
:1008A00010D00523B370033BF370002C08DB737882
:1008B000802040421843C0B201212C4B9847D8E712
:1008C0007078F9E70423B3707178002203920492E0
:1008D000002C09DB843B0B43DAB203A8027201232C
:1008E0004372234B9847C4E70F220A40F5E7012FD4
:1008F0000AD0022F1DD0032F2CD042011A4B9B1877
:1009000006229A70DA70ACE7174B42019918022060
:10091000C870D35C002B05D06201134B9B180522D5
:100920009A709EE702228A70002128000F4B984798
:1009300097E70D4B420199180420C870D35C002B37
:1009400005D06201084B9B1801229A7089E70223A7
:100950008B708EE74201044B9B1800229A7005327F
:10096000DA707EE7C10700001C000020B919000002
:10097000891B0000F0B5C64600B505001F4B98471F
:100980000600430108331E4CE418043421002800FB
:100990001C4B9847C0B208280CD0012128001A4CE3
:1009A000A047802040422843C0B20121A04704BC98
:1009B0009046F0BD00212800134B984698478027A9
:1009C0007F422F43FFB200213800C04772010C4B19
:1009D0009B1801229A705B69210028009847002823
:1009E000E5D17601064B9E190523B370012128003D
:1009F000054CA04701213800A047D8E7C1070000F7
:100A00001C000020111B0000B919000010B5124B8A
:100A1000984700281EDB802200211048104B984781
:100A200000220AE051010D4B5B18FF2159700D495E
:100A300059619961D9610132D2B2032AF2D90A49C6
:100A400000200A4CA0470A490120A047094902207A
:100A5000A047002010BDC046151900001C00002052
:100A60002F1E0000FD07000075090000611D000039
:100A70000108000031080000002800D100BE7047C6
:100A80000368002B03D08B4203D01B68F9E70020DA
:100A900070470120FCE7000070B504000D00064B14
:100AA000984701235840C0B239220449044B984763
:100AB00023682B60256070BD810A0000741E000051
:100AC000790A000003680B60016070470368002B1F
:100AD00003D01A680260180070470020FCE700008D
:100AE00010B5074B5A685A60064B9847064B984713
:100AF0000220064CA047064B9847FD20A04710BD9A
:100B000000400041710B0000410F0000150B000078
:100B10008D0F0000C30709D5114B802252009A6047
:100B2000104A5A600E4B5B78DB09FBD1830709D56D
:100B30000B4B0222FF329A600B4A5A60084B5B78DB
:100B4000DB09FBD1430709D5054B812252009A608E
:100B5000064A5A60024B5B78DB09FBD17047C046FE
:100B6000000C004000070100010501000200010027
:100B7000064B1A7AD2B21A725A7AD2B25A729A7A48
:100B8000D2B29A72DA7AD2B2DA72704700040040B6
:100B900010B50400C3681B7ADB0706D50368002B79
:100BA00000D09847E36801221A7210BD70B50400A6
:100BB0000D00431E9841C0B233221049104B984794
:100BC000E56001232B80AB7ADB09FCD1E268937AE4
:100BD000DB09FCD180331380937ADB09FCD1E26816
:100BE00093698023DB009361937ADB09FCD10133A5
:100BF000E268D371034B1C60002070BD941E00009E
:100C0000790A00009C0000200020704710B5024BBC
:100C10001868024B984710BD9C000020910B000003
:100C2000024B9C466044800AC0B2704700F8FFBD8A
:100C300070B506000C000800714B98470023002B8C
:100C400000D184E00025002E00D18DE0002C00D1E1
:100C500088E001206B4A6C496C4B9847002D00D10D
:100C6000CBE0E369DB0721D42A786B781B021343BE
:100C7000AA7812041343EA7812061A431C231A4076
:100C8000E3699B07FCD123689B0709D523680221F0
:100C90008B432360E3699B07FCD1E3699B07FCD48A
:100CA000012313432360E3699B07FCD1E369DB075E
:100CB000FCD434602B786A7812021A43AB781B0498
:100CC0001A43EB781B0613431C221340082B4DD00C
:100CD000002C00D18DE0002D00D188E001204C4A8D
:100CE00049494A4B98472B786A7812021A43AB78E5
:100CF0001B041A43EB781B061343464A1340236038
:100D0000E3699B07FCD12B796A7912021A43AB790C
:100D10001B041A43EB791B0613433F4A13408022FE
:100D2000920213436360E3695B07FCD12B7B23735F
:100D30006A7B3023E2542B795B075CD1012333714A
:100D4000AA7BEB7B1B021343F380002070BD0028BD
:100D500002D00133DBB272E71D01EA182F4D3C359A
:100D6000AD1870E7002075E7002073E7002C3CD039
:100D7000002D38D001202A4A2349244B98472B784C
:100D80006A7812021A43AB781B041A43EB781B06ED
:100D90001343204A13402360E3699B07FCD12B795E
:100DA0006A7912021A43AB791B041A43EB791B06CA
:100DB00013431C4A13401C4A13436360E3695B07F7
:100DC000FCD12B7A6A7A12021A43AB7A1B041A43BB
:100DD000EB7A1B06134363626A7B3023E254E369B8
:100DE000002BFCD1A7E70020C5E70020C3E70020C7
:100DF00075E7002073E70223A1E70D204042A5E735
:100E0000210C000025090000FC1E0000790A0000EA
:100E1000EF080000FCFEFFFFBF1DFDFFAC1E000041
:100E200003090000BFDDFDFF40020200F0B5CE4621
:100E3000474680B589B081460D0004680B6803936E
:100E40004B6804930023059306930679002814D079
:100E5000002C10D00120374A3749384B9847E369B6
:100E60005B0764D1E3699B07FCD123689B0720D40F
:100E70001420404256E00020EDE70020EBE700227E
:100E80002DE04878000247460743B84602310391F7
:100E9000013205924246A2625BB2002B35DB002094
:100EA00000283ADB0598AB68984202D3069A934231
:100EB00033D9237EDBB25A07E1D5A16A049A002A0E
:100EC00008D0501C04901170012E03D9901C04907E
:100ED000090A5170069A0192013206920122002AF3
:100EE000DAD10699059A9142D6D34946C888D907DE
:100EF000D2D50399002906D0481C03900878804673
:100F0000012EBED8C4E78046C2E701235B4263835B
:100F10008133237613204042C2E7237E9B07FCD017
:100F20000323237609B00CBC90469946F0BD0420FB
:100F30004042F7E7850A0000FC1E0000790A000025
:100F4000104B06229A82104A1A829A6902210A4399
:100F50009A611A7F1D310A401A770A4BDB689B079A
:100F6000FBD5084A938A80210B439BB29382054BA1
:100F7000DB68DB07FBD5034A138A802109010B4399
:100F80001382704700080040060400008222D2014C
:100F90001C4B5A8002221C4B9A841B4BDB68DB06DD
:100FA000FBD51A4A184BDA62194B1B689B0E3F2B74
:100FB00020D09B02802292001343134A936246235F
:100FC0009384938C5B0718D50F4BDA68D0231340BA
:100FD000D02BF9D10C4A938C80210B439BB2938484
:100FE000084B5B78DB09FBD1074A936902218B43ED
:100FF00093617047FC23DB01DFE7034BDB68DB0613
:10100000FBD5E7E7000C004000080040B905FF7D74
:101010002460800000207047124B1A68530B1F2178
:101020000B40900C0140D00D072202401F2B12D024
:101030001F2912D0072A12D09B010B43120313431E
:10104000094A1385D37803210B43D370D3780C213D
:101050000B43D37070471A3BEAE70239EAE7023ADA
:10106000EAE7C046246080000050004170B5837CF0
:101070000F221340C17C083A0A40012A0DD01A0001
:101080000832520119498C4662441021D1715B012A
:10109000174A94466344197070BD4A060CD5C27C49
:1010A00040218A43C2741A00083252010F4CA446F0
:1010B0006244802414715171C27C08218A43C27435
:1010C0000C495A018C180025A572A57608335B01DE
:1010D000064CA44663446F24DC71054B9C46624475
:1010E00014708B6E807C9847D6E7C0460050004154
:1010F00008510041A000002010B5827C0F2313404E
:1011000020228A40D2B25B0105498C4663441A70A2
:10111000044B1B6F8268807C0121984710BDC0463C
:1011200008510041A000002010B5837CFF2B02D0A5
:10113000C27C520600D410BDC27C4024A243C274BB
:10114000024A146F82681800A047F4E7A00000204C
:10115000F0B583B0847C0F232340184D2E8801AD59
:101160002E80FF2C1ED0C47C64061BD500291BD00A
:101170001C0008346401124DAC466444802525717E
:1011800001AD6E5C1C00083464010D4FBC46644424
:10119000E671695C5B010B4CA44663441970110055
:1011A000094B984703B0F0BD1C0008346401044D9E
:1011B000AC46644440256571E2E7C046181F000054
:1011C000005000410851004129110000F0B583B0E2
:1011D000837C0F2213403C4A948801AA14805A0150
:1011E0003A4CA418002933D01A0008325201384D65
:1011F000525D120907251540C27C072616400A01D8
:10120000A218947AE4B2022D2AD0A40744D5947A85
:101210000225AC43947201AC655C1A00083252019D
:101220002B4FBC466244D571625C5B01294CA446DD
:1012300063441A70012E45D1C37C5B0642D5C37C42
:10124000DB0999423ED000221900234B984739E030
:101250001A00083252011E4D555D07221540CBE79A
:10126000E507D2D5947A0125AC43947201AC655C54
:101270001A0008325201164EB4466244D571625CBF
:101280005B01144CA44663441A704B1E9941C9B2C9
:101290000422114B984715E05A00521812010B48CE
:1012A00082180020907201A8445C1A000832520192
:1012B000074DAC466244D471425C5B0105498C46E3
:1012C00063441A7003B0F0BD181F0000A000002096
:1012D00000500041085100415111000070B5002537
:1012E00018E0104C6034AE007319980010302018CC
:1012F000043003210C4B984772199300E3182633EE
:10130000FF221A707619B300E418273400232370E3
:101310000135EDB2082DE4D9602200210148034BCC
:10132000984770BDA0000020291100002F1E00006A
:10133000F0B5C64600B505000E00837C0F241C40A6
:101340006201564B9B18002958D059698904890CB1
:101350002B8A534A934253D0013B1BB20B40EA7C89
:1013600007271740002E07D02200083252014D48AF
:10137000844662440220D071AA6894466144A96000
:101380006A6891424ED292B28BB2D21A92B2EB7C80
:101390009B0637D52B8A98469A4200D890462B68F0
:1013A0009C4661444246E8683F4B9847E9686201C1
:1013B0003A4B9B1819616301384AD2185169434668
:1013C0009B049B0C890B89030B4353615169374B79
:1013D0000B405361002E07D1012F5DD04A226301DB
:1013E00033498C4663441A70083464012D4B9C4683
:1013F00064448023637104BC9046F0BD0021A7E7DC
:101400001BB2ABE780239B019A4207D890462B681A
:1014100059186201214B9B181961CCE780239B016D
:101420009846F4E7EA7CD2060FD5EB7C1022934372
:10143000EB746201194B9B185A69920B9103596125
:1014400059691A4A0A405A61C4E7012F0DD0640154
:10145000184A944664444A2222702A8A93420BD046
:1014600000212800144B9847C5E76401114A9446AF
:1014700064444B222270F0E7EB7C40229343EB74F0
:10148000064BDB6EA87CA96898470028B3D1EB7C9B
:1014900040221343EB74E3E74E22A0E7A0000020B4
:1014A000FF030000005000411D1E0000FF3F00F040
:1014B000095100410851004129110000F8B5DE46EC
:1014C00057464E464546E0B504000F00837C0F2585
:1014D0001D40002959D06A01714B9B185B681B01A4
:1014E0009B0C9A46002F53D06A016D4B9B185B688A
:1014F0009B049B0C9846268A6A4B9E4201D0013E73
:10150000B6B2434633409B46E37C07221A409146DD
:10151000002F07D02B0008335B01634A94466344D5
:101520000122DA71E37C9B0611D56268002A0ED095
:1015300092B22389D21A92B22368A1688C4663447E
:101540001800E168934500D25A46584B98476368A3
:10155000002B20D1E27CD2061DD5E37C10229343E0
:1015600020221343E3744E496A01E3685350238AEF
:101570008A1851689B041B094D4801400B43536076
:1015800053689B0B9903516047E000239A46A9E7F3
:1015900000239846AFE7002F1DD0228A93451AD228
:1015A000E37C10229343E374A3684344A3604B4657
:1015B000012B66D06B013F4A9446634425221A7082
:1015C000002D03D16D01364BE268EA500021200066
:1015D000394B984733E0A2685244A2609342E6D95F
:1015E0009BB291B25B1A9BB2E17C89062DD5218A10
:1015F0008B4200D81900E0686B01294A98506B01B2
:101600002748C01842688B041B0929490A40134324
:10161000436043689B0B9A034260002F08D14B46FE
:10162000012B35D025226B0124498C4663441A7066
:1016300008356D011C4B9C46654440232B713CBC16
:1016400090469946A246AB46F8BD218A8B420BD9FB
:10165000802189018B420FD8B343190023689A185F
:101660006B010F481A50CAE78B4208D2E17C202058
:101670000143E1741900F1E780218901EEE71900C7
:10168000ECE76B010B4A944663442D221A7097E7EE
:101690006A01034B9B1800229A762D32C3E7C0469D
:1016A000A0000020FF030000005000411D1E0000AC
:1016B000FF3F00F00851004129110000095100418D
:1016C00070B5894B1D8CADB2002D01D00024BFE058
:1016D000998B1B8B0B405A070DD49A0515D41A060B
:1016E00037D470221A423ED11A0757D4DB0700D5EF
:1016F00068E0002306E004227B4B9A837B4B1B6E41
:1017000098470123002BE1D070BD774B784A9A832C
:101710009A82923AFF3A1A830023012B12D8580179
:10172000724A121812891207120F032A02D00133CB
:10173000DBB2F2E76D4B1B1819894904490D0022F1
:101740001A8100E00021694B5B6E0320984701235A
:10175000D8E78022644B9A83644B5B6E002105209E
:1017600098470123CEE7604B9A839A82604A1A8396
:10177000604B9B8C9B060CD45E4BDA68D0231340E5
:10178000D02BF9D1594B5B6E0021022098470123E1
:10179000B8E7584BDB68DB06FBD5F3E7524B00217B
:1017A000802252009954F83A9A8368329A82504AB9
:1017B0001A83514B98474D4B5B6E0021012098478F
:1017C00001239FE7484B4A4A9A839A82923AFF3A0A
:1017D0001A83464B5B6E002104209847012391E752
:1017E000DA0607D45A0608D49B062FD50021434BAE
:1017F00098472BE0424B984728E001213F4B984700
:1018000024E05A060FD41A0711D49A0713D4C17CC6
:1018100007220A40012A19D15A0710D4DB0615D530
:10182000374B984712E00121344B98470EE00121D5
:10183000344B98470AE00121334B984706E00021DA
:10184000304B984702E000212C4B98470134E4B21A
:10185000082C00D958E7254B6033A20011198800E5
:1018600001001030181804305B1826331B78FF2B4A
:10187000ECD0827C0F23134001229A402A42E5D00B
:101880001A000832520118498C466244D2795B0131
:101890001E498C4663441B781340D7D0C27C472135
:1018A000114001299CD052B2002AAADB9A06CAD460
:1018B0005A070DD4DA070FD4C17C07220A40012A47
:1018C000C4D11A070CD4DB06C0D50D4B9847BDE731
:1018D00000210C4B9847B9E701210D4B9847B5E71C
:1018E0000121084B9847B1E700500041A0000020BB
:1018F0000102000000080040DD120000F9100000A5
:101900006D100000CD11000031130000095100419D
:10191000BD14000000B583B0002201AB5A70214B0A
:101920009B78DB071BD41F4B9B789B07FBD11D4B80
:101930001B789B070CD51B4A137802218B4313702D
:10194000184B9B789B07FBD1164B9B789B07FBD4CE
:101950000122144B1A70134B9B789B07FBD1114B40
:101960009B78DB07FBD4104B104A1A665A669A66BE
:10197000DA661A670E4B98470E4B98470422094BBC
:101980001A70084B9B789B07FBD1064A064B5362A3
:1019900001AB5B7801210B43DBB21381002003B064
:1019A00000BDC04600500041A000002015100000FE
:1019B000DD12000019100000F0B50F22024040B205
:1019C000C40F002A05D0002801DB130002E0931C9D
:1019D00000E013001D009800C018830010331800A9
:1019E000474B60331B180433022A00D984E00129D5
:1019F00018D000293DD0AA0052199100404B603305
:101A00005B1826331A780F23134008335B013D4AD5
:101A10009446634498791023A3401840431E98418C
:101A2000C0B2F0BD364803006033AA005619B100B9
:101A30005B1826331B780F210B401026A640F6B208
:101A40001900083149012F4FBC4661444E712021D5
:101A5000A140CCB259012C4B9C4661440C705219E8
:101A60009300C3188033DA7908210A43DA71002021
:101A7000D7E79A7C0F310A4011000831490121480B
:101A80008446614488791021A140084224D0C9B21B
:101A9000100008304001604401712021A140CEB205
:101AA00055011A4FBC4665442E70C07908420AD0D1
:101AB000110008314901134884466144CE71012068
:101AC000A040C0B20871D87C07210140012905D08F
:101AD000DA7C08218A43DA740020A2E70832520136
:101AE00008498C466244917930221142F4D10200B7
:101AF00008218A43DA74EFE71220404291E7C0469A
:101B0000A00000200050004109510041085100414F
:101B100070B50E000F2404406201184B9B18196821
:101B20005D68AD04AD0C022C1FD8002E20D0230020
:101B300008335B01124A9B5C112B1CD12300083334
:101B40005B0194466344DB79DB0601D4002070BD61
:101B5000082230000B4B984708346401084B9C4620
:101B600064441023E3712800F1E712204042EEE7BD
:101B700012204042EBE713204042E8E7A00000209B
:101B8000005000411D1E0000F0B5DE4657464E468F
:101B90004546E0B585B08046057A0F222A406DB2F1
:101BA000EB0F9946002A05D0002D01DB100002E062
:101BB000901C00E010000600614B603381000F189C
:101BC000BC0010341C190434B8001B189B8C5D49F0
:101BD0008B4244D05F1EBFB2414649680F40022A83
:101BE00000D9A3E042461268574882420CD98818AF
:101BF0000190564884460198604505D8920703D164
:101C0000002D2EDB99422FD2B200921991004C4B3D
:101C10005B1880331B68002B00D18AE001230193FD
:101C2000002D0BDB002F09D0B20092199100444B1C
:101C30005B1880331B68002B00D17DE0B200921945
:101C400091003F4B5B188033DB791B070FD50220D7
:101C500005B03CBC90469946A246AB46F0BD1F007D
:101C6000BAE700230193DBE700230193D8E703A839
:101C7000374B9847B20092199100314B5B18803373
:101C8000DB795B0630D4B3009B199A002C4B9B4642
:101C9000934480235B449A46DB79402213435246A7
:101CA000D37103A82B4B98475B46424612685A678C
:101CB000424652689A6700235A46D3674B46DB0177
:101CC0005246D2797F211140019A52010B432021C3
:101CD0008B431A435346DA7143465B7A002B08D094
:101CE000002F1BD0002205E003A81A4B98470120C3
:101CF000AEE70022B3009E19B100114B5B18803390
:101D00001101DA79102082430A43DA71002D07DBD2
:101D100000212000104B9847002099E70122E9E7B5
:101D2000002120000D4B9847002091E712204042EF
:101D30008EE7132040428BE71220404288E7C046DE
:101D4000A0000020FF030000FFFFFF1FFF0F002087
:101D50008D0500009B050000BD140000311300003C
:101D6000002908D0002808D0012809D0022806D16F
:101D7000054B196703E00549F4E7034B9966704783
:101D8000014BD966FBE7C046A000002015100000FB
:101D900010B5014B984710BDC116000010B50B4B94
:101DA000984700230EE00A4AD15C4A091F200840E8
:101DB00001218140D201C020C00584466244916166
:101DC0000133DBB2072BEED9FEE7C0461501000058
:101DD000441F000070B500260C4D0D4C641BA41070
:101DE000A64209D1002600F0B7F80A4D0A4C641B40
:101DF000A410A64205D170BDB300EB589847013638
:101E0000EEE7B300EB5898470136F2E7641F000095
:101E1000641F0000641F0000681F0000002310B54D
:101E20009A4200D110BDCC5CC4540133F8E70300E2
:101E30008218934200D1704719700133F9E700000E
:101E40002E2E2F68616C2F7372632F68616C5F7325
:101E500070695F6D5F73796E632E63002E2E2F683D
:101E6000616C2F7372632F68616C5F74696D65724A
:101E70002E6300002E2E2F68616C2F7574696C73B1
:101E80002F7372632F7574696C735F6C6973742E32
:101E9000630000002E2E2F68706C2F7274632F6801
:101EA000706C5F7274632E6300000000000000001D
:101EB0000000000000000000000000000000000022
:101EC0000000000000000000000000000000000012
:101ED0000000000000000000000000000000000002
:101EE00000000000000000000C00200000000200C4
:101EF00000000000FE00FF01000000002E2E2F68F1
:101F0000706C2F736572636F6D2F68706C5F736593
:101F100072636F6D2E630000254A00000408000004
:101F200048020020000000004000000008020020DD
:101F30000000000040000000C80100200000000078
:101F4000400000001211100908070B0A0B0A0000DC
:101F50000908070012111000F8B5C046F8BC08BC0B
:101F60009E467047DD000000F8B5C046F8BC08BCCE
:081F70009E467047B500000019
:00000001FF
